:10000000000000308A00422BFF00030E8301A10094
:100010007F08A0000A08A8008A01A00E0408A20018
:100020007708A3007808A4007908A5007A08A6003C
:100030007B08A700831383128C308400001C2228C5
:100040000C183B288C308400801C28288C183D28F4
:10005000220884002308F7002408F8002508F90086
:100060002608FA002708FB0028088A00210E8300D2
:10007000FF0E7F0E09008A11E0288A11E3280A107A
:100080008A100A1182074834413443344B342034F7
:10009000763431342E343034003400340A108A106F
:1000A0000A1182070A340D340A340D3425347334AE
:1000B00000340A108A100A11820725344C34753432
:1000C0006534343420342B34203425344C347534A6
:1000D000203447344F3400340A108A100A11820742
:1000E00025344C3475346534343420342B34203486
:1000F00025344C347534203452344534503445342E
:10010000413454342034253475340A340D340034E9
:100110000A108A100A11820725344C34753465346C
:10012000343420342B34203425344C34753420348A
:100130004834413443344B3400340A108A100A11D5
:10014000820725344C3475346534343420342B34F0
:10015000203425344C347534203474346934633499
:100160006B34733400340A108A100A118207253464
:100170004C347534203478342034313420347034A5
:10018000723465347334633461346C3465340034F0
:100190000A108A100A1182074534723472346F349F
:1001A000723400340A108A100A11820725344C3444
:1001B000753420347434693463346B3473340034EC
:1001C0000C108A1128288C108A11282842308400AB
:1001D000831300080319FD280130F800BF30F70031
:1001E0006400F70BF028F80BEE284A30F700F70B05
:1001F000F72800006400800BEC2800348316861179
:10020000831286110830F800000000000000F81783
:100210001829F813CC0C03188615031C86117817BF
:1002200018297813F80B0A29000000000000861531
:100230000130F7008401840B1B29F70B1A290D30BC
:100240008400840B212900000000F81B0929781B79
:10025000112900340408F8000830F7008316061549
:100260008312061D352983163029C101F717482945
:10027000F7134829031006190314C10C77174829EE
:100280007713F70B3A29780884004108F8005D29B4
:10029000013084000030F71B5530F800F80B4E2970
:1002A000840B4A290D30F71B0330F800F80B562950
:1002B000F71B3829771B40293A298A11C12BCB011A
:1002C0000408CA004B10831B4B14440EF038C600C0
:1002D000C607E23EC700323EC90044080F39C707CF
:1002E000C707C907E93EC800C807C807430E0F394A
:1002F000C807C907C80DC90DC909C90D43080F3979
:10030000C907C60D0730C5000A30C907C803031C5A
:100310008529C807C703031C8929C707C603031C0F
:100320008D29C607C503031C91294530840083131A
:1003300007304A058407493004020319C12900081F
:10034000F700031DA9294A1ABF29CA19AB29203071
:10035000AC290830CA003030F707C4010408C300D4
:100360004410831B44147708C5007708CC00FE2096
:10037000430884008313441883174508F700840A50
:100380009B290008F7003030F7077708CC00FE20E3
:1003900000344708F80146020318D1294608F7003F
:1003A000DD29F7010830C800C60DF70D47087702B0
:1003B0000318F700F80DC80BD42900344513C512F3
:1003C0004408C6006430C700C9217708C400780813
:1003D000031D082AC51A082AC519162A451BF6291D
:1003E0004518F6294519F629C51B162A451C022A67
:1003F000C51B162A451B022A4518162A4519022A2A
:10040000C51B162A2030451E3030CC00FE20162A8F
:10041000C516C51F122A78088000F8002D30CC00C0
:10042000FE20C51330307807CC00FE20451B212A62
:100430004408C6000A30C700C9217708C400451720
:10044000E729C51F262A2D30CC00FE203030440776
:10045000CC00FE208A118F2C1030F700FA01CD015C
:10046000CA0CC90C031C3A2A4B08FA070318CD0A18
:100470004C08CD07CD0CFA0CF90CF80CF70B302A10
:100480008A11B62AC701C5010A30C600C401C301DA
:1004900041084204031D502A0030F800F900412BA6
:1004A0004708C70A410784008313421883170008CE
:1004B000C80048082D3C031D692A0130C5004708C3
:1004C000C70A410784008313421883170008C80035
:1004D000762A48082B3C031D762A4708C70A41079D
:1004E00084008313421883170008C80048082F3C73
:1004F0000318322B4808393C031C322B4808303C87
:10050000031DA22A4708410784008313421883175A
:100510000008783C0319962A470841078400831392
:10052000421883170008583C031DA22A1030C60049
:10053000C70A4708C70A4107840083134218831774
:100540000008C80046080A3C031DC92A48082F3C79
:100550000318C82A4808393C031CC82ACA010A30B3
:10056000C9004408CC004308CB002C2A3030480294
:100570007807C3007908C4000318C40A4708C70AEB
:10058000410784008313421883170008C800A62A75
:10059000322B4608103C031D322B4808603C0318E0
:1005A000D82A48087A3C031CD82A4808DF39D92AB7
:1005B0004808C80048082F3C0318E22A4808393C7C
:1005C0000318EA2A4808403C0318322B4808463CE6
:1005D000031C322B48082F3C0318072B4808393CD2
:1005E000031C072B430DC900440DCA00C90DCA0DD9
:1005F000C90DCA0DC90DCA0DF030C9053030480209
:100600004907C3004A08C4000318C40A1C2B430D41
:10061000C900440DCA00C90DCA0DC90DCA0DC90DC6
:10062000CA0DF030C905413048020A3E4907C300EF
:100630004A08C4000318C40A4708C70A41078400CF
:100640008313421883170008C800603C03182F2B3F
:1006500048087A3C031C2F2B4808DF39302B480808
:10066000C800DA2A46080A3C031D3D2B450B3D2BEA
:10067000C309C409C30A0319C40A4308F80044089B
:10068000F9000034840183131F30830583161F1281
:100690009F121B0880399B0007309C0005086400EE
:1006A0001C0883120D13603083168F00861183128D
:1006B0008615A901AA010130AB00AC01AD01AE0164
:1006C00083161F129F121B0880399B0083121F1074
:1006D00094128316061186140612003083129400B9
:1006E000831694000108C7392838810087308312A7
:1006F00090000030F800920000308316920007301E
:100700009C00050864000230F700F70B852B000001
:1007100000001C0883120D1383169D0162308F00A8
:1007200064308312C200E620C10141084E20C10A94
:10073000F700CC00FE2004304102031D952BC201BE
:1007400042083F2000380319A92BC20ACC00FE2022
:10075000A02B8316061283120612831686128312AA
:100760008612BF010130BE00BD01BC010A30CC00C1
:10077000FE200D30CC00FE203E30CC00FE20C0011B
:100780002A297808B1003108CC00FE204008C00AB0
:10079000323E840083133108800031080D3C031978
:1007A000D52B4008093C0318C02B32304007840089
:1007B000831380010A30CC00FE200D30CC00FE20D7
:1007C0003208673A0319F12B153A0319602C1A3ACB
:1007D0000319E92C013A0319712D193A0319A82DAF
:1007E000EB2D103084003D08C4003C08C3005F219D
:1007F0000330C10041085920C10AF700CC00FE2097
:1008000008304102031DFA2B103084003F08C40059
:100810003E08C3005F212030CC00FE204730CC00D2
:10082000FE204F30CC00FE20B001AF0130083D0269
:10083000031C3C2C031D202C3C082F0203183C2CCD
:100840008F018E010F08FA000E08F7000F087A02D8
:10085000031D222C7708C1007A08C2004208273CF9
:10086000031C382C031D222C41080F3C0318222C9A
:10087000AF0A0319B00A162C8F018E010F08FA0077
:100880000E08F7000F087A02031D3E2C7708C100FE
:100890007A08C20042083F02031C542C031D3E2C60
:1008A0003E084102031C3E2C8316061283120616D4
:1008B0000130C200E62083160612831206121A2E99
:1008C000C0014008C00AC100103084003D08C400C7
:1008D0003C08C3005F210330C20042086C20C20AFA
:1008E000F700CC00FE2008304202031D6D2C1030B2
:1008F00084003F08C4003E08C3005F210B30C300E2
:1009000043086C20C30AF700CC00FE2013304302DA
:10091000031D802C4108C4001830C500DE290A30B0
:10092000CC00FE200D30CC00FE20B001AF0130081D
:100930003D02031CBD2C031DA12C3C082F020318F3
:10094000BD2C8F018E010F08FA000E08F7000F086A
:100950007A02031DA32C7708C1007A08C20042085E
:10096000273C031CB92C031DA32C41080F3C031882
:10097000A32CAF0A0319B00A972C8F018E010F0820
:10098000FA000E08F7000F087A02031DBF2C770843
:10099000C1007A08C20042083F02031CD52C031D87
:1009A000BF2C3E084102031CBF2C83160612831283
:1009B00006161430C200E6208316061283120612B1
:1009C0000830C100FA30C200E620C10BE22C612CD5
:1009D0001A2E103084003D08C4003C08C3005F217B
:1009E0000330C10041088820C10AF700CC00FE2076
:1009F00008304102031DF22C103084003F08C4006F
:100A00003E08C3005F210B30C20042088820C20AA2
:100A1000F700CC00FE2010304202031D052DB0016E
:100A2000AF0130083D02031C372D031D1B2D3C0870
:100A30002F020318372D8F018E010F08FA000E08C0
:100A4000F7000F087A02031D1D2D7708C1007A08F0
:100A5000C2004208273C031C332D031D1D2D4108F5
:100A60000F3C03181D2DAF0A0319B00A112D8F0179
:100A70008E010F08FA000E08F7000F087A02031D16
:100A8000392D7708C1007A08C20042083F02031CD2
:100A90004F2D031D392D3E084102031C392D8316AD
:100AA00006128312061683160613831206130A30E3
:100AB000C200E62083168612831286162830C100F3
:100AC000FA30C200E620C10B602D83168612831215
:100AD00086128316061283120612831606178312D5
:100AE0001A2EC10141083F20003803197B2DC10A8D
:100AF000CC00FE20722D0A30CC00FE200D30CC0040
:100B0000FE20103084003D08C4003C08C3005F2173
:100B10000330C10041089D20C10AF700CC00FE202F
:100B200008304102031D8A2D103084003F08C400A4
:100B30003E08C3005F210B30C20042089D20C20A5C
:100B4000F700CC00FE2011304202031D9D2D1A2E0D
:100B500033082F3C0318DF2D3308393C031CDF2DED
:100B6000C2013330C10042227908BD007808BC00C0
:100B7000103084003D08C4003C08C3005F210330EE
:100B8000C1004108B320C10AF700CC00FE200730A5
:100B90004102031DC12D0430C2003030CC00FE20C4
:100BA000C20BCD2D0730C3004308B320C30AF700A2
:100BB000CC00FE2010304302031DD42DEA2DC101CC
:100BC0004108C820C10AF700CC00FE2005304102D0
:100BD000031DE02D1A2E32082F3C03180F2E320869
:100BE000393C031C0F2EC2013230C1004222790869
:100BF000BF007808BE00103084003F08C4003E08E3
:100C0000C3005F210330C1004108D220C10AF700B0
:100C1000CC00FE2009304102031D042E1A2EC10112
:100C20004108C820C10AF700CC00FE20053041026F
:100C3000031D102EB62B83160612831206120230E5
:100C4000C1009630C200E620C10B212E8316061289
:100C5000831206160230C1009630C200E620C10B96
:060C60002C2E1B2E322E8B
:04400E003137FC3F0B
:00000001FF
